:100000000C94C2060C94EA060C94EA060C94EA06D8
:100010000C94EA060C94EA060C94EA060C94EA06A0
:100020000C94EA060C94EA060C94EA060C94EA0690
:100030000C94EA060C94EA060C94EA060C94EA0680
:100040000C9498120C94EA060C94EF1B0C94C91BA8
:100050000C94EA060C94EA060C94EA060C94EA0660
:100060000C94EA060C94EA06FF08180936094F09B1
:10007000810968099A099A09030B050B030B050B03
:10008000030B050B030B050B05100D1015101F10AE
:100090002510251041105310FD29042A712A402AE9
:1000A000712A192A712A5E2A712A232A4A2A712A58
:1000B000692A0D2A712A122A2D2A712A712A712A77
:1000C000712A712A712A662A712A712A712A712A63
:1000D000712A712A712A712A712A712A712A452A74
:1000E000712A1E2A712A712A712A282A148018005E
:1000F0000009021202120212021202120209140173
:10010000120310050E070C090A0B080D060F041147
:100110000209280902120212021202120212020934
:1001200000000008000201000003040700000000B6
:100130000000000015EF03038002CF0300C130ED83
:100140000464031281E803850078CB05392C003460
:1001500002F70120EA020000C00123C10110C5021C
:100160003E28C701863601483A0155B1020018B64B
:1001700003088227F20100260101E00F0F312B0C4A
:100180000E084EF1370710030E0900E10F000E14A0
:1001900003110731C148080F0C31360F118078293F
:1001A000000F001C0000FE00FFF9FFF3FFE7FFCF88
:1001B000FF9FFF3FFE7FFCFE0004000FE7FF87FE6E
:1001C00007F807E00780060007F3FFE7FFCFFF9F70
:1001D000FF3FFE7FFCFC01F807F00F001C00FE0152
:1001E000F803F3FFE7FFCFFF9FFF3FFE7FFCFE001A
:1001F00006001E007E01FE07FE1FFE7F00020007B4
:10020000F3FFE7FFCFFF9FFF3FFE7FFCFFF9FFF00B
:1002100007F00015801E00001302130213021302E0
:1002200013021302130213020C0205020C02050250
:100230000C090C090C02130213020F0103020D0337
:1002400003020B050302072A040503020502060345
:100250000302050208010A02130213021302130229
:1002600013021302130215801E000213021302135D
:10027000021302130213021302130205020C0205F9
:10028000020C090C09130213021302130206010CDB
:100290000204030C020205052C05020205050205F5
:1002A00002040305020D01050213021302130213D7
:1002B00002130213021317002200FFFFF9FFFFF3DE
:1002C000FFFFE7FFFFCFFFFF9FFFFF3FFFFE7FFF27
:1002D000FCFE6001FCC003F99FFFF33FFFE7FFFF57
:1002E000CFFBFF99C7FF320FFE6001FCC003F990FE
:1002F00067F338CFE7FD9FCFFF3F99FE7F33FC00C8
:10030000600000C003FFFFE7FFFFCFFFFF9FFFFF7D
:100310003FFFFE7FFFFCFFFFF9FFFFF01700220009
:100320003FFFFE7FFFFCFFFFF9FFFFF3FFFFE7FF4B
:10033000FFCFFFFF9FFFFF000CFE0019FFFF33FF01
:10034000FE67FFFFCFFFBF9FFC733FE0E67F800C9F
:10035000FE0019FC0733F98E67F3DFCFE7FF9FCF6D
:10036000F33F9FE67F000C00001800FFFFF9FFFF3E
:10037000F3FFFFE7FFFFCFFFFF9FFFFF3FFFFE7F82
:10038000FFFC15001E00FFFFE7FFFF3FFFF9FFFF27
:10039000CFE7FC7F3FC7F9FC7FCFC7FE7C7FF3C769
:1003A000FF9C7FFCC7FFE47FFF07FC007FE003FFAB
:1003B000FE0FFFF23BFF989FFCE07FE783FF380FC3
:1003C000F9807FCF01FE7E0FF3FC3FFFF9FFFFCFE7
:1003D000FFFE7FFFF015001E003FFFF9FFFFCFFF7C
:1003E000FE7FFFF1FF3FC7F9FF1FCFFC7E7FF1F3D8
:1003F000FFC79FFF1CFFFC67FFF13FFFC1FFFF002E
:100400001FFC00FF93FFF09FFE0CFFC067FC073F3F
:10041000F039FF83CFF81E7F8DF3F8FF9FCFFFFEEB
:100420007FFFF3FFFF9FFFFC18000E00FDFFFFF8AA
:10043000FF1FF07F1FE03F1FC01F1F800F1F00071F
:100440001FF8E000F8F001F8F803F8FC07F8FE0FD9
:10045000F8FF1FFFFFBF0F0420080000000000008E
:10046000000000000000000000000370F870FF7042
:10047000F80700E000FC00E0000000E000FC00E005
:100480000A00113011C013003D00D13011C013001B
:100490003D00D1001107607830FC108EF8FF108706
:1004A000F0C3E06110007E00FF0081108120FF405A
:1004B0007E8001000200040018E027F04F10881031
:1004C00008F00FE0070EE001E003F003307C10FEBF
:1004D000908FD08FE0F1E070F004300730062004F8
:1004E00040000300E000FC00E005E007F81F0C30CE
:1004F0000240018005018002400C30F81FE0070730
:100500000060006C00AC00F000AC006C0060090002
:1005100002000200020002E03F00020002000200AE
:1005200002037200740038000580008000800080A3
:1005300000800003700070007000053000C00100F2
:100540000E0070008008801FE07FF0FF1080108098
:10055000F0FFE07F801F0710201060F07FF07FF039
:10056000FF10001000091000306070C0B0C030E310
:1005700030FE307C30384000086020704030C410BD
:10058000CE10FFE0F7E073C001088003800580090A
:100590008011F07FF0FFF0FF800108600C707C306C
:1005A000DC30DC10DE10CE20CFC08308C007E01F97
:1005B000F03F3078104CF0CFE087C0830800600037
:1005C000C000C030C0C0C000C700F800C008E07064
:1005D000F07910FE108E108FF08FE0FBC0710810C4
:1005E0003C107E30FF2083E0C1C0FF807F003E03CF
:1005F000701C701C701C03721C741C381C0A0004D4
:10060000000A000A000A00110011802080208020CA
:10061000404009000900090009000900090009001B
:1006200009000900090A4040802080208020001134
:100630000011000A000A000A00040800700070702F
:10064000B07083708400FC00F8007011E007180C93
:1006500004300220E241F147F18F119E6190F18F49
:10066000F19F119F12502260C430081F10000D101E
:1006700000100070009003800C803080FC907FF0B0
:100680001FF003F000300010000C10801080F0FF0D
:10069000F0FFF0FF10841084108430CEF0FFE07B78
:1006A000C0310C800FC03FE07F706030C010801000
:1006B00080108010801040206040F00D108010806D
:1006C000F0FFF0FFF0FF10801080108030C06060FD
:1006D000E07FC03F800F0C10801080F0FFF0FFF033
:1006E000FF10841084109F108010C030E0F0000BC9
:1006F00010801080F0FFF0FFF0FF10841084009F46
:10070000008000C000E00E800FC03FE07F607030CE
:10071000C01080108010811081F041E061E0F10094
:100720000100010E10801080F0FFF0FFF0FF108438
:10073000000400041084F0FFF0FFF0FF1080108030
:100740000710801080F0FFF0FFF0FF108010800A8B
:10075000E000E000D00010801080F0FFE0FFC0FF5C
:10076000008000800E10801080F0FFF0FFF0FF107E
:10077000841086800FD013F0A170A030C0108010BC
:10078000800B10801080F0FFF0FFF0FF10801080D1
:10079000100010003000F0001210801080F0FF10E8
:1007A000C010F000FE803FE00FF001C00100061015
:1007B0003810C0F0FFF0FFF0FF108010800E100026
:1007C0001080F0FF10F01078003C001E000F800732
:1007D000C083E081F0FF008000800D000FC03FE08B
:1007E0007F606030C010801080108030C06060E09A
:1007F0007FC03F000F0B10801080F0FFF0FFF0FF74
:100800001082108200C600FE007C00380D800FC0F0
:100810003FE07F706030C018801C801E8036C07240
:1008200060E27FC23F800F0E10801080F0FFF0FF6B
:10083000F0FF108210838083C0C7E0FC707C3038EA
:100840001000100009F039607C20FC108E1086101A
:1008500087F043E0F3C0010B00E0008010801080BF
:10086000F0FFF0FFF0FF10801080008000E00D002E
:10087000800080C0FFE0FFF0FF308010801000108B
:10088000802080C0FF008000800D008000C000F04C
:1008900000FC80BFE08FF00360008003008C00B09C
:1008A00000C0008013008000C000F000FC00BFE02A
:1008B0008FF003E080008300EC00F800FFE09FF081
:1008C00003E0000007009800E000800D1080108019
:1008D00030C050F090F800BF000FD00FF091F0A0A2
:1008E00030C0108010800D008000C000F010F810A3
:1008F000BEF08FF007F0031004109800A000C000B5
:10090000800C100030F0F0C0F081D087108F10BE46
:1009100010F810F010C03080F00004FFFFFFFF015E
:100920008001800500C000380007E00010000401CD
:10093000800180FFFFFFFF09000400180020004035
:10094000008000400020001800040A01000100019E
:10095000000100010001000100010001000100038D
:10096000D00A00C0006009600EF00EF01690112051
:1009700011F01FF01FF00F1000090080F0FFE0FFE2
:10098000E0FF10081010F01FE00FC00707C007E0DD
:100990000FF01F30101010101C200C09C007E00FC2
:1009A000F01F10102088F0FFF0FFE0FF200007C0CC
:1009B00007E00FF01F3012101E100E200607101057
:1009C000F07FF0FFF0FF109000C000C009360779FB
:1009D0000FB91FB910B910B91F391F3A161C100AE8
:1009E0001080F0FFF0FFF0FF10080010F01FF01F64
:1009F000F00F1000051010F0DFF0DFF0DF10000640
:100A0000060007000110FFDFFFDFFEDF0B1080F0A4
:100A1000FFF0FFF0FF10018003D013F01C701830BE
:100A2000101000051080F0FFF0FFF0FF10000F1015
:100A300010F01FF01FF01F10080010F01FF01FF043
:100A40000F10080010F01FF01FF00F10000A101018
:100A5000F01FF01FF01F10080010F01FF01FF00F24
:100A6000100008C007E00FF01F10101010F01FE07A
:100A70000FC007090110FF1FFF1FFF1F21081010E3
:100A8000F01FE00FC00709C007E00FF01F10102192
:100A900010FF1FFF0FFF1F0100081010F01FF01FB5
:100AA000F01F10080010001C001C06700E201F9084
:100AB00017D013F009E01C060010E01FF03FF0FF14
:100AC000101020100A0010E01FF01FF01F1000206F
:100AD00010F01FF01FF01F1000090010001C801FF5
:100AE000E01FF01360008013001C00100E001000C7
:100AF0001C001FE01FF013E0000017001EE01FF0B5
:100B000017E0000017001800100910101010301C1A
:100B1000501FC01FF003F014301810100906100702
:100B200018071E821FEC17F0018013001C0010082C
:100B30001000701CF010F013901F101F301C70106C
:100B40000500018C32FE7E73CC018001FFFF0501A0
:100B50008073CCFE7E8C3200010A00030004000486
:100B60000004000200020001000100010006000074
:100B7000000000250028002B0000000000240027B2
:100B8000002A000404040404040404020202020211
:100B90000203030303030301020408102040800141
:100BA000020408102001020408102007012003009D
:100BB000000001FA03C000C00528FE28FE28052415
:100BC00052FF4A2406626408102646055CA2520CB5
:100BD0001201C0027E8102817E02C0C00508083E6B
:100BE000080801030508080808080102030638C0C0
:100BF000047C82827C0240FE04468A926204448223
:100C0000926C041868FE0804F4A2A29C047C9292E0
:100C10004C04808EB0C0046C92926C046492927CFE
:100C200001120113030814220314141403221408DC
:100C300004408A9060083C4299A5B985443806066C
:100C400038C8C8380606FE929292926C067C828260
:100C500082824406FE828282827C05FE9292928289
:100C600005FE90909080067C828292945E06FE1033
:100C7000101010FE01FE040C0202FC05FE102844B8
:100C80008204FE02020208FEC0300C0C30C0FE06D8
:100C9000FEC0300C02FE067C828282827C06FE90C0
:100CA00090909060067C82828A867D06FE9090906D
:100CB000906E05649292924C058080FE808005FCC7
:100CC000020202FC05C0380638C007C03806180604
:100CD00038C005C6281028C605C0201E20C00586BD
:100CE0008A92A2C202FF8103601C030281FF0340BB
:100CF000804005020202020202804004042A2A1EE9
:100D000004FE22221C041C222214041C2222FE04A3
:100D10001C2A2A18027E90041925253E04FE102064
:100D20001E01BE0201BF04FE18240201FE073E2080
:100D3000203E20201E043E20201E051C2222221CB4
:100D4000043F242418041824243F023E2004122ABD
:100D50002A24027C22043C02023E0438060638059E
:100D600038061806380336083603310A3C03262AAB
:100D70003203083641017F034136080420402040F9
:100D80000000DF2B11241FBECFEFD8E0DEBFCDBFA8
:100D900012E0A0E0B1E0E8EEFBE502C005900D92A4
:100DA000A431B107D9F722E0A4E1B2E001C01D925D
:100DB000AD3EB207E1F716E0C2ECD6E004C02197E1
:100DC000FE010E94A22DC13CD107C9F70E946D28E7
:100DD0000C94F22D0C9400008EE480937C0062E071
:100DE00070E080E090E00E94521280917A0080646E
:100DF00080937A0080917A0086FDFCCF8091780004
:100E00002091790030E0322F2227A901330F660BA1
:100E1000770B9A01AB01282B64EB7BE281E190E038
:100E20000E94832DCA01B9010895CF93DF9300D0AA
:100E300000D0CDB7DEB7BE016F5F7F4FCE01039606
:100E40000E9497130F900F900F900F90DF91CF910A
:100E50000895EF92FF920F931F93CF93DF937C013E
:100E6000EB018A0197FF07C08DE291E00E942219F1
:100E7000F194E194F108C7016AE070E00E944D2D01
:100E80009B017C01A801BE01C9010E94C418A801F0
:100E9000BE018FE291E00E942219A801BE01C701A4
:100EA000DF91CF911F910F91FF90EF900C94C41898
:100EB000DF92EF92FF920F931F93CF93DF93D82E81
:100EC0000AE010E0C0E0D0E083E2E82EF12C8D2DA6
:100ED0000E943B12C80FD91FF7013197F1F701505B
:100EE0001109A9F7CE016AE070E00E944D2DCB01F7
:100EF000DF91CF911F910F91FF90EF90DF900895B8
:100F00003F924F925F926F927F928F929F92AF9299
:100F1000BF92CF92DF92EF92FF920F931F93CF93E6
:100F2000DF93CDB7DEB728970FB6F894DEBF0FBEBC
:100F3000CDBF382E6801662349F02901032E000C2D
:100F4000660877084A01821A930A0AC02701421AE2
:100F5000530A052C000C660877084901841A950A83
:100F6000092C000CAA08BB0880914902332029F003
:100F7000882349F081E391E004C0882321F084E3D1
:100F800091E00E94F22680914902882391F0A3010A
:100F9000920160E87AE186E090E00E943D2D20E039
:100FA00034E840E050E00E94832DCA01B9010E945C
:100FB000672680914902882321F087E391E00E940F
:100FC000F226A0E4B1E0A30192010E94C62D20E028
:100FD00034E040E050E00E94832D29013A0129834A
:100FE0003A834B835C83A0E0B6E9A50194010E949B
:100FF000C62D20E034E840E050E00E94832D80912F
:101000004902882361F0CA01B9012D833E834F83D1
:1010100058870E94672658854F813E812D81809197
:101020004902882361F087E391E02D833E834F835B
:1010300058870E94F22658854F813E812D81A0EF6E
:10104000B0E00E94C62D2CE03EEF4FEF5FEF0E9414
:10105000832D49015A018FEE880E911CA11CB11CF1
:1010600090EF89169104A104B1042CF06FEE862E46
:10107000912CA12CB12C80914902882349F085E064
:10108000A82FAC9DC001AD9D900D11240E94E026BB
:10109000332079F07201EE0CFF1CF0921802E092FE
:1010A0001702C401880F991F9093160280931502AE
:1010B0006FC0E0901702F0901802F7FE03C0BFEF78
:1010C000EB1AFB0AF594E794E40CF51CF092180275
:1010D000E0921702809115029091160297FD0196F9
:1010E00095958795880E991E90921602809215020A
:1010F000F7FE03C02FEFE21AF20AF594E794C70156
:101100000F2C000CAA0BBB0B89839A83AB83BC8387
:1011100097FE03C09FEF891A990A3401759467946A
:101120004301072C000CAA08BB086091470270918C
:1011300048020FEF1FEF9301A701809145029091A4
:1011400046020E94601E80914502909146028135C0
:101150009105F4F4A1E5EA16F104D4F0B4EE6B16AF
:101160007104B4F480914E0290914F0297FF08C031
:1011700070921A0260921902D0924D02C0924C02F3
:1011800070924F0260924E02D0924B02C0924A027D
:1011900089819A81909346028093450290924802F9
:1011A0008092470228960FB6F894DEBF0FBECDBFDF
:1011B000DF91CF911F910F91FF90EF90DF90CF9033
:1011C000BF90AF909F908F907F906F905F904F9067
:1011D0003F90089580E592E00E941D1B892BD1F37A
:1011E00080E592E00E94FB1A0895019788309105EE
:1011F00008F0BDC08C5C9F4FFC010C94A22D8CE8C4
:1012000090E090934402809343028FE090E09093AB
:1012100042028093410240EE5FEF66E574E089E3AD
:1012200091E00E94221920EE3FEF45ED53E018C0F7
:101230008BE890E090934402809343028FE090E02B
:10124000909342028093410240EE5FEF66E574E0C6
:1012500082EF91E00E94221920EE3FEF42E853E036
:1012600069E170E082E990E00C94842088E790E0E6
:1012700090934402809343028FE090E09093420267
:101280008093410240EE5FEF66E574E08DE391E00C
:101290000E94221920EE3FEF4CE153E0E1CF88E7B6
:1012A00090E090934402809343028FE090E090930B
:1012B00042028093410240EE5FEF66E574E086E40F
:1012C00091E00E94221920EE3FEF46EB52E0C8CF9A
:1012D00082E890E090934402809343028FE090E094
:1012E000909342028093410240EE5FEF66E574E026
:1012F0008FE491E00E94221920EE3FEF43E152E09B
:10130000AFCF82E890E090934402809343028FE055
:1013100090E0909342028093410240EE5FEF66E5D9
:1013200074E086E591E00E94221920EE3FEF46E648
:1013300052E096CF88E890E0909344028093430275
:101340008FE090E0909342028093410240EE5FEF85
:1013500066E574E08DE591E00E94221920EE3FEFF2
:101360004CEE50E069E170E086E990E07DCF85E6E3
:1013700090E090934402809343028FE090E090933A
:1013800042028093410240EE5FEF66E574E083E63F
:1013900091E00C94221908958EBD00000DB407FE53
:1013A000FDCF8EB508958CBD9DBD0895CF93DF937D
:1013B000C82FD62F80E590E00E94D30960E08AE034
:1013C0000E94EF118C2F82958F708D2B0E94CC097B
:1013D0008C2F8295807F0E94CC0961E08AE0DF91AA
:1013E000CF910C94EF11CF93DF93EB0160E10E945A
:1013F000D6091C161D0644F4BE01DD0F880B990B9F
:10140000DF91CF910C945212DF91CF910895CF9339
:10141000DF93EB0160E90E94D6091C161D0644F417
:10142000BE01DD0F880B990BDF91CF910C94521206
:10143000DF91CF9108952F923F924F925F926F92DA
:101440007F928F929F92AF92BF92CF92DF92EF9254
:10145000FF920F931F93CF93DF93CDB7DEB72897FB
:101460000FB6F894DEBF0FBECDBF8C019B015A01B1
:1014700061E070E0822F2D833E830E94070A2D8158
:101480003E81A4EEBFEF0E94A82D6B017C01950167
:10149000A8E1BCEF0E94A82DA7019601260F371FD7
:1014A000481F591F29833A834B835C8328EE33E01E
:1014B000D5010E94BF2D4B015C013FEF3F834FEFF1
:1014C000488722242A94322C9EEDC92EDD24D39401
:1014D000E12CF12C412C512C32014A9460E1809195
:1014E00000010E94D60982E090E00E945807053072
:1014F000110571F426E730E0DC010E94BF2D29813F
:101500003A814B815C81620F731F841F951F09C054
:101510009C01AAE8BFEF0E94A82D680D791D8A1DC5
:101520009B1DA70196010E94832D209300013093FB
:1015300001014093020150930301809100019091B9
:101540000101A0910201B0910301B7FF08C0109200
:10155000000110920101109202011092030180918A
:10156000000190910101A0910201B09103018F3F10
:101570009105A105B10549F044F040920001509257
:10158000010160920201709203018091000190912B
:101590000101A0910201B09103012816390629F03A
:1015A0002F8038848F83988799CF0197A109B1093B
:1015B00021E08E3F9105A105B10508F020E0822FC2
:1015C00028960FB6F894DEBF0FBECDBFDF91CF9146
:1015D0001F910F91FF90EF90DF90CF90BF90AF9051
:1015E0009F908F907F906F905F904F903F902F9043
:1015F000089501978830910570F4845C9F4FFC0139
:1016000060E10C94A22D80E008C08FEF0E94D60903
:1016100060E980E006C060E18FEF0E94D60960E9D2
:101620008FEF0C94D609CF92DF92EF92FF920F9337
:101630001F93CF93DF938C010E94F90A03301105A9
:1016400009F49DC024F40130110554F413C1043091
:10165000110509F45CC0073011050CF4CAC00AC1B9
:1016600020914A0230914B0280914C0290914D02A0
:1016700082179307DCF5C8010E94F5084FEF57E089
:1016800066E574E080E791E00E942219A0911902BA
:10169000B0911A0280914E0290914F02A81BB90B93
:1016A00020E137E20E94BF2D20914A0230914B0287
:1016B00040914C0250914D02241B350B032E000C1F
:1016C000440B550B0E94832DCA01B90120EF30E075
:1016D00040E050E00E94832DDA01C901E9014FEF9B
:1016E00057E066E574E00E94C418C6C080914902C4
:1016F000882309F4D8C087E791E0DF91CF911F914B
:101700000F91FF90EF90DF90CF900C94F42684E03F
:1017100090E00E94F5084FEF57E066E574E08BE734
:1017200091E00E94221961E070E080E80E94070ABF
:1017300000E010E0C0E0D0E09AE0C92ED12CC80152
:10174000B6010E944D2D862F6AE070E00E94F309D9
:1017500080E090E00E9458077C0181E090E00E94C8
:101760005807E81AF90A8BE0E816F1040CF07AC081
:1017700021960B5E1F4FC536D10509F771C083E076
:1017800090E00E94F5084FEF57E066E574E08BE7C4
:1017900091E00E94221961E070E080E80E94070A4F
:1017A00000E010E0C0E0D0E086EFC82EDD24DA943F
:1017B000C801B6010E944D2D862F6AE070E0845268
:1017C0000E94F30982E090E00E9458077C0183E0C8
:1017D00090E00E945807E81AF90A8BE0E816F10435
:1017E0000CF040C021960B5E1F4FC536D10501F7A6
:1017F00037C0C8010E94F5084FEF57E066E574E076
:1018000081E891E00E9422190530110549F44FEF5B
:1018100057E066E574E08DE291E00E94221902C073
:1018200006E010E0C0E0D0E0AE0160E870E0C80182
:101830000E941B0A882381F082E090E00E945807F2
:101840008C0183E090E00E945807081B190B1016CA
:10185000110644F405E010E02196C536D10521F7C4
:10186000C0E0D0E04FEF57E066E574E0CE010E94A3
:10187000290702C0C0E0D0E080914902882321F00E
:1018800088E891E00E94F22680914902882359F06D
:10189000CE01DF91CF911F910F91FF90EF90DF90DC
:1018A000CF900C94E026DF91CF911F910F91FF9084
:1018B000EF90DF90CF9008952F923F924F925F92DA
:1018C0006F927F928F929F92AF92BF92CF92DF9250
:1018D000EF92FF920F931F93CF93DF93CDB7DEB7B5
:1018E0002A970FB6F894DEBF0FBECDBF5C017A8792
:1018F00069875E834D834901059739F43FEF3A8349
:101900004EEF242E33243A9404C01A8232E0232E60
:10191000312C87E090E00E9458072C0188279927F6
:10192000881999099C838B8369847A847194619462
:10193000710829853A858D819E81821793070CF461
:1019400094C06EE170E08A810E94070ACA80D12C9F
:1019500019828FEFC816D10411F008F046C04985EE
:101960005A85B601C5010E941B0A8823D1F195E072
:10197000A916B104D1F482E090E00E9458079C01BE
:1019800083E090E02F8338870E9458077201098511
:101990001A852F813885AC0160E0898191E0892723
:1019A0000E94800721E029831DC081E090E00E9411
:1019B00058079C0180E090E02F8338870E945807E9
:1019C000EE24EA9423E0F22E09851A852F813885CA
:1019D000AC0161E0898186270E94800731E039836C
:1019E00001C01982C20CD31CB4CF809147029091E0
:1019F0004802029620914502309146022E5F3F4FE9
:101A00003093440220934302909342028093410218
:101A10004FEF5FEF6BEA7BE095E0A916B10411F49C
:101A2000C30102C089859A850E9429074FEF5FEFA5
:101A30006BEA7BE08BE891E00E94221980914902D9
:101A4000882321F08DE891E00E94F4260E9415077A
:101A50002B813C81620E731E811122C089859A857B
:101A6000880D991D9A87898764CFC5012A960FB67C
:101A7000F894DEBF0FBECDBFDF91CF911F910F91C4
:101A8000FF90EF90DF90CF90BF90AF909F908F909E
:101A90007F906F905F904F903F902F900C94130B1E
:101AA0002A960FB6F894DEBF0FBECDBFDF91CF915F
:101AB0001F910F91FF90EF90DF90CF90BF90AF906C
:101AC0009F908F907F906F905F904F903F902F905E
:101AD00008952F923F924F925F926F927F928F92D2
:101AE0009F92AF92BF92CF92DF92EF92FF920F93AD
:101AF0001F93CF93DF93CDB7DEB760970FB6F894FF
:101B0000DEBF0FBECDBF4C01762E642E1901188B9F
:101B10000F87FA86E9862601BC86AB868FEF9FEF9A
:101B200090934F0280934E0210924D0210924C02FD
:101B300010924B0210924A0280914902882321F0B0
:101B40008FE891E00E94F42685E0849D9001859DB8
:101B5000300D11243A832983429CA001439C500DEF
:101B6000529C500D11245C834B834F855889429DB4
:101B70009001439D300D529D300D112438872F83E5
:101B8000849F9001859F300D11243E832D83212C4D
:101B9000312CA12CB12C2F85388949855A854217C3
:101BA00053070CF4ABC04F855889452B41F460E1D5
:101BB000872D0E94D609CC24CA94D12C37C08F819E
:101BC0009885820D931D6AE070E00E944D2D862F4E
:101BD000860D80931B0260E1ECCF82E090E00E94D2
:101BE00058079C0183E090E02D873E870E945807AC
:101BF000AC0181E02D853E859FEFC916D10409F027
:101C000080E0EB84FC840F85188960E00E948007E7
:101C1000809147029091480297FF03C0CC24CA9458
:101C2000DC2C22E0C21AD108D7FC10C061E070E0C1
:101C30008C2D0E94070A5FEFC516D10471F66EE184
:101C400070E080E090E00E945212C7CF4F85588923
:101C500014161506C4F520914502309146022E5FF8
:101C60003F4F3093440220934302029690934202E6
:101C70008093410251E08516910499F083E0881623
:101C8000910409F54FEF5FEF6BEA7BE08F85988950
:101C90000E9429074FEF5FEF6BEA7BE08BE891E052
:101CA00010C04FEF5FEF6BEA7BE08D819E818A0D64
:101CB0009B1D0E94C4184FEF5FEF6BEA7BE081E948
:101CC00091E00E94221980914902882321F08DE839
:101CD00091E00E94F4260E94150729813A81A20E04
:101CE000B31E4B815C81240E351E811122C08F856D
:101CF0009889840D951D988B8F874DCFC401609670
:101D00000FB6F894DEBF0FBECDBFDF91CF911F910C
:101D10000F91FF90EF90DF90CF90BF90AF909F908A
:101D20008F907F906F905F904F903F902F900C948A
:101D3000130B60960FB6F894DEBF0FBECDBFDF91D8
:101D4000CF911F910F91FF90EF90DF90CF90BF90B8
:101D5000AF909F908F907F906F905F904F903F904B
:101D60002F9008952F923F924F925F926F927F92A1
:101D70008F929F92AF92BF92CF92DF92EF92FF929B
:101D80000F931F93CF93DF9300D000D0CDB7DEB772
:101D90009C838B8387E090E00E9458075C010E943F
:101DA000402682E090E090934402809343028CEEC0
:101DB00090E0909342028093410240E154E86BEA44
:101DC0007BE089E791E00E94221900E114E820EF0E
:101DD00030E040E050E060E070E080E090E00E94A1
:101DE000601E2FEE30E040E451E06FEE70E080E0E6
:101DF00090E00E94601EC12CD12C7601C3948B818F
:101E00009C818D7F9A838983A4E8B0E0A701960125
:101E10000E94C62D25E030E040E050E00E94832D76
:101E200019012A01C901029690934402809343024A
:101E3000EDEEF0E0F0934202E093410289819A8155
:101E4000019721F0EB81FC81369741F440E154E8A1
:101E50006BEA7BE08DE291E00E94221940E154E8B8
:101E60006BEA7BE0C6010E94C41840E154E86BEACB
:101E70007BE08BE891E00E94221900E114E820EF5A
:101E800030E0A10160E070E0C1010E94601EFFEF40
:101E9000CF1ADF0AEF0AFF0A8DE0C816D104E10469
:101EA000F10409F0B1CF25E0C22ED12CE12CF12CA8
:101EB000A0EFB0E0A70196010E94C62D2EEC3FEFE7
:101EC0004FEF5FEF0E94832D19012A019FEE290E2B
:101ED000311C411C511CE2E0F0E0F0934402E0931D
:101EE0004302C10108969093420280934102898186
:101EF0009A81019721F0EB81FC81369741F440E112
:101F000054E86BEA7BE08DE291E00E94221940E107
:101F100054E86BEA7BE0C6010E94C41840E154E833
:101F20006BEA7BE084E991E00E94221900E114E869
:101F3000910140E451E0B10180E090E00E94601E18
:101F4000F5E0CF0ED11CE11CF11C87E3C816D104CB
:101F5000E104F10409F0ACCF8B819C810E94F5086B
:101F6000EB81FC81E530F105C4F4E330F105CCF4FC
:101F7000319754F1809132029091330225E030E0A4
:101F8000B9010E944D2D4B018091140190911501D2
:101F9000B9010E944D2D3B0117C08B819C81079791
:101FA0009CF420913002309131028AE0829F4001FE
:101FB000839F900C11242091120130911301829F74
:101FC0003001839F700C1124C301881999098D3346
:101FD000910544F48F31910544F445974CF421E088
:101FE00030E008C02AE030E005C025E030E002C063
:101FF00022E030E0EB81FC813197E830F10508F018
:1020000061C0EC5BFF4F0C94A22D69017301840148
:1020100025EE3FEF47ED50E03FC079018301940189
:102020004BE150E06EE070E049C06901730184014A
:102030002BEE3FEF4CED50E06CED70E02FC07901DE
:102040008301940145E150E037C0A301B4018B81C5
:102050009C810F900F900F900F90DF91CF911F9167
:102060000F91FF90EF90DF90CF90BF90AF909F9037
:102070008F907F906F905F904F903F902F900C9437
:102080005C0C9AE0C92ED12CE12CF12C00E010E080
:1020900020E030E04FEF50E06FEF70E08B819C81EB
:1020A0000E94690D0FC08AE0E82EF12C00E010E0DC
:1020B00020E030E040E050E060E070E08B819C8107
:1020C0000E9402270F900F900F900F90DF91CF91F9
:1020D0001F910F91FF90EF90DF90CF90BF90AF9046
:1020E0009F908F907F906F905F904F903F902F9038
:1020F0000895BF92CF92DF92EF92FF920F931F93BA
:10210000CF93DF93EC01B62E9091140281E08927E2
:1021100080931402209771F420913402309135029B
:102120002230310539F4811103C0C6E0D0E002C08D
:10213000C5E0D0E0C530D10551F0C630D10571F40D
:1021400060E180E00E94D60960E98FEF0DC060E198
:102150008FEF0E94D60960E980E006C060E180E868
:102160000E94D60960E980E80E94D6098FE1C82E56
:10217000D12C61E070E080E090E00E945212C33008
:10218000D10561F02CF4C230D10508F044C006C07E
:10219000C530D10519F0C730D105E9F582E00E94BC
:1021A0003B128C0183E00E943B127801E81AF90A85
:1021B00083E3E816F1047CF1BB20C1F0C530D10502
:1021C000A9F06EE170E08FEF0E94F30983E00E94B6
:1021D0003B128C0182E00E943B12081B190B0E0D72
:1021E0001F1D0233110514F4C7E0D0E081E090E038
:1021F0000E94F90A209709F063C0809134029091FF
:1022000035028130910509F459C0029711F485E037
:102210005AC081E058C0C430D10571F03CF4209719
:1022200059F0C230D10509F042C006C0C630D10510
:1022300019F0C830D105D9F580E00E943B128C011D
:1022400081E00E943B127801E81AF90A83E3E8165C
:10225000F1046CF1BB20C1F0C530D105A9F06EE1ED
:1022600070E080E00E94F30981E00E943B128C0143
:1022700080E00E943B12081B190B0E0D1F1D02333C
:10228000110514F4C8E0D0E082E090E00E94F90A61
:102290002097B1F4809134029091350281309105FC
:1022A00089F0029711F486E00EC082E00CC081E054
:1022B000C81AD10809F05DCF80E005C083E003C0F3
:1022C000CE0102C084E090E0DF91CF911F910F9189
:1022D000FF90EF90DF90CF90BF9008953FB7F894B4
:1022E0008091220290912302A0912402B0912502B4
:1022F00026B5A89B05C02F3F19F00196A11DB11D61
:102300003FBFBA2FA92F982F8827820F911DA11D9B
:10231000B11DBC01CD0142E0660F771F881F991FD8
:102320004A95D1F70895FC018081918120853185FE
:102330002817390724F4318320839187808784818B
:102340009581208531852817390724F43583248326
:102350009187808782819381268137812817390769
:1023600024F433832283978386838081918124811F
:1023700035812817390724F431832083958384839A
:1023800086819781208531852817390724F4378382
:1023900026839187808782819381248135812817C4
:1023A000390724F433832283958384838081918148
:1023B000268137812817390724F4318320839783B6
:1023C000868384819581268137812817390724F4F3
:1023D000358324839783868384819581089590E053
:1023E000FC01E05EFE4F3491FC01E956F44F24916C
:1023F000FC01ED57F44FE491EE2309F43BC0332385
:1024000039F1333091F038F43130A9F0323001F540
:1024100084B58F7D12C0373091F03830A1F0343060
:10242000B9F4809180008F7D03C0809180008F7708
:10243000809380000DC084B58F7784BD09C08091E2
:10244000B0008F7703C08091B0008F7D8093B00083
:10245000F0E0EE0FFF1FE159F44FA591B4918FB753
:10246000F894EC91611103C020952E2301C02E2B0E
:102470002C938FBF08958E3008F08E508770806443
:1024800080937C0080917A00806480937A008091B0
:102490007A0086FDFCCF809178002091790090E051
:1024A000922B08958F929F92AF92BF92CF92DF921C
:1024B000EF92FF926B017C010E946E114B015C0157
:1024C000C114D104E104F104F1F00E946E11DC01A9
:1024D000CB0188199909AA09BB09883E9340A10537
:1024E000B10570F321E0C21AD108E108F10888EEC5
:1024F000880E83E0981EA11CB11CC114D104E10414
:10250000F10419F7DDCFFF90EF90DF90CF90BF90EF
:10251000AF909F908F9008952FB7F89460911E020E
:1025200070911F0280912002909121022FBF089587
:102530001F920F920FB60F9211242F933F938F93F8
:102540009F93AF93BF9380911E0290911F02A09121
:102550002002B091210230911D0223E0230F2D377C
:1025600020F40196A11DB11D05C026E8230F029697
:10257000A11DB11D20931D0280931E0290931F0286
:10258000A0932002B0932102809122029091230215
:10259000A0912402B09125020196A11DB11D809346
:1025A000220290932302A0932402B0932502BF91AC
:1025B000AF919F918F913F912F910F900FBE0F90F0
:1025C0001F901895CF93CFB7F89480911C0281117A
:1025D00024C0EDE8FBE08491E1EAFBE09491E82F70
:1025E000F0E0EE0FFF1FE758F44FA591B491EC9186
:1025F000E92321F461E08AE00E94EF118AE00E9461
:102600004E288CB580618CBD8CB580648CBD8DE00E
:102610000E944E288BE00E944E2880911C028F5F02
:1026200080931C02CFBFCF91089560E08091060196
:102630000E94EF1160E0809107010E94EF118AE291
:102640008EBD00960096009601D001C0089561E00D
:10265000809106010E94EF111EBC000000960096BA
:1026600001D001C0089510922C0210922B021EBCC2
:102670000000009601D001C008958091170190914B
:102680001801019790932A02809329029EBD00961B
:102690000096009601D001C00895809129028EBD58
:1026A00000000096009601D001C0089560E080917E
:1026B00006010E94EF118BE28EBD009600960096F7
:1026C00001D001C0089561E0809106010E94EF11E0
:1026D0001EBC00000096009601D001C00895109223
:1026E0002E0210922D021EBC0000009601D001C0E7
:1026F00008958091190190911A01019790932802F1
:10270000809327029EBD00960096009601D001C0DE
:102710000895809127028EBD00000096009601D09A
:1027200001C0089561E0809107010C94EF118F9230
:102730009F92AF92BF92CF92DF92EF92FF920F9350
:102740001F93CF93DF93CDB7DEB764970FB6F8949E
:10275000DEBF0FBECDBF6C017B0182E591E00E9420
:10276000D30960E0809108010E94EF118BE8A82E48
:10277000BB24B394C5010197F1F784EB90E00E946C
:10278000372384EB90E00E9437234C0184EC90E0E7
:102790000E9437238C0181E990E00E94372381E970
:1027A00090E00E94372323E0969587952A95E1F7DC
:1027B0009C878B8781E990E00E94372333E09695D0
:1027C00087953A95E1F79E878D8781E990E00E9491
:1027D000372343E0969587954A95E1F7988B8F8745
:1027E00081E990E00E94372353E0969587955A95AA
:1027F000E1F79A8B898B81E990E00E94372363E0AF
:10280000969587956A95E1F79C8B8B8B81ED90E08F
:102810000E94372381ED90E00E94372373E0969564
:1028200087957A95E1F79A83898381ED90E00E94FC
:102830003723E3E096958795EA95E1F79C838B83B0
:1028400081ED90E00E943723F3E096958795FA9505
:10285000E1F79E838D8381ED90E00E943723A3E012
:1028600096958795AA95E1F798878F8381ED90E0FB
:102870000E943723B3E096958795BA95E1F79A873A
:10288000898780E090E00E94372361E08091080111
:102890000E94EF11F5013197F1F70E94CB0980E515
:1028A00091E00E94D3090E94CB0983E0969487941B
:1028B0008A95E1F793E0169507959A95E1F7080D4B
:1028C000191D013811050CF48FC380910901823064
:1028D00009F4CCC0833009F4BDC1813009F09DC238
:1028E00000910E0110910F01CE010B960E949311E1
:1028F000D801A81BB90B2091170130911801009144
:102900000E0110910F010E94BF2D209110013091F6
:102910001101A801421B530B9A01032E000C440B1A
:10292000550B0E94832DCE010B9657FD26C00E94A9
:102930009311D801A81BB90B2091170130911801F0
:102940000E94BF2D20910E0130910F014091100186
:1029500050911101241B350B032E000C440B550B19
:102960000E94832DCA01B9010E94B12C20E030E001
:1029700040E05FE30E940D2C25C00E949311D80116
:10298000A81BB90B20911701309118010E94BF2D8F
:1029900020910E0130910F014091100150911101D1
:1029A000241B350B032E000C440B550B0E94832D6A
:1029B000CA01B9010E94B12C20E030E040E05FE3A1
:1029C0000E940C2C0E94792CF60171836083009187
:1029D0000A0110910B01CE0101960E949311D801BA
:1029E000A81BB90B2091190130911A0100910A011D
:1029F00010910B010E94BF2D20910C0130910D010F
:102A0000A801421B530B9A01032E000C440B550BDB
:102A10000E94832DCE01019657FD14C00E94931190
:102A2000D801A81BB90B2091190130911A010E94FD
:102A3000BF2D20910A0130910B0140910C01509162
:102A40000D01ADC10E949311D801A81BB90B2091B3
:102A5000190130911A010E94BF2D20910A01309175
:102A60000B0140910C0150910D01BFC100910E016D
:102A700010910F01CE0101960E949311D801A81B5D
:102A8000B90B209117013091180100910E0110919E
:102A90000F010E94BF2D2091100130911101A8015A
:102AA000421B530B9A01032E000C440B550B0E9442
:102AB000832DCE01019657FD26C00E949311D801A7
:102AC000A81BB90B20911701309118010E94BF2D4E
:102AD00020910E0130910F01409110015091110190
:102AE000241B350B032E000C440B550B0E94832D29
:102AF000CA01B9010E94B12C20E030E040E05FE360
:102B00000E940D2C25C00E949311D801A81BB90B5F
:102B100020911701309118010E94BF2D20910E01C4
:102B200030910F014091100150911101241B350B80
:102B3000032E000C440B550B0E94832DCA01B901D2
:102B40000E94B12C20E030E040E05FE30E940C2CBA
:102B50000E94792CF6017183608300910A01109123
:102B60000B01CE010B960E949311D801A81BB90B43
:102B70002091190130911A0100910A0110910B0165
:102B80000E94BF2D20910C0130910D01A801421B24
:102B9000530B9A01032E000C440B550B0E94832DFE
:102BA000CE010B9657FD27C00E949311D801A81B98
:102BB000B90BC0901901D0901A0196010E94BF2D47
:102BC00020910A0130910B0140910C0150910D01AF
:102BD000241B350B032E000C440B550B0E94832D38
:102BE000CA01B9010E94B12C20E030E040E05FE36F
:102BF0000E940D2C26C00E949311D801A81BB90B6E
:102C0000C0901901D0901A0196010E94BF2D209109
:102C10000A0130910B0140910C0150910D01241BD0
:102C2000350B032E000C440B550B0E94832DCA015B
:102C3000B9010E94B12C20E030E040E05FE30E9447
:102C40000C2C0E94792CC61AD70AF701D182C082B7
:102C500081E0D1C1CE010B960E94931140911001E9
:102C600050911101DC01A41BB50B2091170130918B
:102C700018010E94BF2D20910E0130910F01241BDD
:102C8000350B032E000C440B550B0E94832DCE01F7
:102C90000B9657FD26C00E94931140911001509150
:102CA0001101DC01A41BB50B209117013091180113
:102CB0000E94BF2D20910E0130910F01241B350B76
:102CC000032E000C440B550B0E94832DCA01B90141
:102CD0000E94B12C20E030E040E05FE30E940D2C28
:102CE00025C00E9493114091100150911101DC0107
:102CF000A41BB50B20911701309118010E94BF2D24
:102D000020910E0130910F01241B350B032E000C76
:102D1000440B550B0E94832DCA01B9010E94B12CAE
:102D200020E030E040E05FE30E940C2C0E94792C10
:102D3000F60171836083CE0101960E949311409148
:102D40000C0150910D01DC01A41BB50B2091190160
:102D500030911A010E94BF2D20910A0130910B0180
:102D6000241B350B032E000C440B550B0E94832DA6
:102D7000CE01019657FD26C00E94931140910C018F
:102D800050910D01DC01A41BB50B2091190130916C
:102D90001A010E94BF2D20910A0130910B01241BC2
:102DA000350B032E000C440B550B0E94832DCA01DA
:102DB000B9010E94B12C20E030E040E05FE30E94C6
:102DC0000D2C25C00E94931140910C0150910D01D2
:102DD000DC01A41BB50B2091190130911A010E944E
:102DE000BF2D20910A0130910B01241B350B032EBE
:102DF000000C440B550B0E94832DCA01B9010E949F
:102E0000B12C20E030E040E05FE30E940C2C0E94F7
:102E1000792CF701718360831BCFCE0101960E944C
:102E200093114091100150911101DC01A41BB50BCD
:102E300020911701309118010E94BF2D20910E01A1
:102E400030910F01241B350B032E000C440B550B46
:102E50000E94832DCE01019657FD26C00E9493113A
:102E60004091100150911101DC01A41BB50B209180
:102E70001701309118010E94BF2D20910E01309151
:102E80000F01241B350B032E000C440B550B0E9425
:102E9000832DCA01B9010E94B12C20E030E040E04E
:102EA0005FE30E940D2C25C00E94931140911001F8
:102EB00050911101DC01A41BB50B20911701309139
:102EC00018010E94BF2D20910E0130910F01241B8B
:102ED000350B032E000C440B550B0E94832DCA01A9
:102EE000B9010E94B12C20E030E040E05FE30E9495
:102EF0000C2C0E94792CF60171836083CE010B9615
:102F00000E94931140910C0150910D01DC01A41B12
:102F1000B50B2091190130911A010E94BF2D20910B
:102F20000A0130910B01241B350B032E000C440BBE
:102F3000550B0E94832DCE010B9657FD27C00E9492
:102F4000931140910C0150910D01DC01A41BB50BB4
:102F50000091190110911A0198010E94BF2D209132
:102F60000A0130910B01241B350B032E000C440B7E
:102F7000550B0E94832DCA01B9010E94B12C20E09B
:102F800030E040E05FE30E940D2C26C00E949311C8
:102F900040910C0150910D01DC01A41BB50B009177
:102FA000190110911A0198010E94BF2D20910A0168
:102FB00030910B01241B350B032E000C440B550BD9
:102FC0000E94832DCA01B9010E94B12C20E030E09B
:102FD00040E05FE30E940C2C0E94792C061B170B2B
:102FE000F7011183008334CEF60111821082F701BC
:102FF0001182108280E064960FB6F894DEBF0FBE97
:10300000CDBFDF91CF911F910F91FF90EF90DF9097
:10301000CF90BF90AF909F908F9008952F923F9246
:103020004F925F926F927F928F929F92AF92BF92D8
:10303000CF92DF92EF92FF920F931F93CF93DF9384
:103040001F92CDB7DEB75A01FB0124913196E4906F
:103050003196E4914E2F50E0E82FF0E0E417F507A9
:1030600008F47EC0FB013396682F70E046175707BF
:10307000B0F46491662309F473C03196203130F0C6
:1030800093E0699FE00DF11D112407C070E0283026
:1030900010F0660F771FE60FF71F8150E5CF049100
:1030A00010E0BF016F5F7F4F822E912CF12C011534
:1030B000110509F44CC0FB014490512C612C712C7A
:1030C0001B01FFEF2F1A3F0A283080F0F1012490F6
:1030D00052281B01F2E02F0E311C203138F0F10193
:1030E000249062281B01F3E02F0E311C8091040113
:1030F000882301F1C12CD12C8C149D04D8F040FE02
:1031000011C060914102709142026E0D7F1D6C19D9
:103110007D09A501809143029091440229830E9478
:10312000761D298176946794579447948FEFC81A37
:10313000D80AE2CF80914302909144020196909385
:1031400044028093430201501109B101B0CF809134
:10315000430290914402019690934402809343026B
:103160000F90DF91CF911F910F91FF90EF90DF9023
:10317000CF90BF90AF909F908F907F906F905F9017
:103180004F903F902F9008958F929F92AF92BF9251
:10319000CF92DF92EF92FF920F931F93CF93DF9323
:1031A000EC016B015A0197FF07C0D195C195D10978
:1031B0008DE20E940E1802C0892B51F085E0E82EA6
:1031C000F12C00E117E220E09AE0892E912C0FC04B
:1031D00080E3DF91CF911F910F91FF90EF90DF90EF
:1031E000CF90BF90AF909F908F900C940E18C01707
:1031F000D10714F4222359F0CE01B8010E944D2DBD
:10320000862FA501B601805D0E940E1821E0CE0137
:10321000B8010E944D2DEC01C801B4010E944D2D52
:103220008B0181E0E81AF10811F7DF91CF911F912E
:103230000F91FF90EF90DF90CF90BF90AF909F9055
:103240008F900895EF92FF920F931F93CF93DF9388
:103250008B017A01EC018991882329F0A701B8013B
:103260000E940E18F8CFDF91CF911F910F91FF9020
:10327000EF9008952F923F924F925F926F927F92BC
:103280008F929F92AF92BF92CF92DF92EF92FF9276
:103290000F931F93CF93DF93CDB7DEB76E970FB623
:1032A000F894DEBF0FBECDBF9C8B8B8B7C876B876A
:1032B0001A013E8F2D8F1E870D87141615060CF0F0
:1032C00043C1121613060CF03FC1449F3001459FC5
:1032D000700C700C1124229FA001239F500D500DE3
:1032E00011245A874987C301072C000CAA0BBB0B7A
:1032F0008F87988BA98BBA8B72E0880F991FAA1FB2
:10330000BB1F7A95D1F78D839E83AF83B8879A01CF
:10331000032E000C440B550B29833A834B835C83AB
:10332000E2E0220F331F441F551FEA95D1F72D8B82
:103330003E8B4F8B588FAD8DBE8DB195A195B10948
:10334000AA0FBB1F1196C980DA80EB80FC80CC0CE1
:10335000DD1CEE1CFF1C93010E94A82DC60ED71E7B
:10336000E81EF91E4B885C8826E030E0A985BA8506
:103370000E94BF2D698F7A8F8B8F9C8F01E010E0A8
:10338000812C912C54019301AD8DBE8D0E94A82DEE
:10339000681579058A059B050CF450C02D853E857E
:1033A000A8016B857C858D8D9E8D681B790BC20174
:1033B0000E943A1D2D853E85A8016B857C85AD8DCB
:1033C000BE8D6A0F7B1FC2010E943A1DF7FC13C01D
:1033D000A1E0B0E0ED8DFE8DAE1BBF0B2D813E81D7
:1033E0004F8158850E94D12DC60ED71EE81EF91EAA
:1033F0003197FE8FED8FD501C40162E0880F991FD0
:10340000AA1FBB1F6A95D1F7298D3A8D4B8D5C8D14
:10341000820F931FA41FB51FC80ED91EEA1EFB1EE4
:1034200089819A81AB81BC81880E991EAA1EBB1E20
:1034300091E0491A51080E5F1F4FA5CFAA27BB275D
:10344000A219B309AA0FBB1F119629853A850E94BC
:10345000A82D0F85188929893A89000F111F221F6D
:10346000331F68017901C60ED71EE81EF91E26E03B
:1034700030E0D3010E94BF2D4B015C01412C512C47
:1034800032011E821D8229853A85D1010E94A82D14
:1034900064157505860597050CF456C08101000F6B
:1034A000111F0F5F1F4F2D853E85A8016B857C8501
:1034B000AD81BE816A1B7B0BEB89FC89E219F309A4
:1034C000FA83E983CF010E943A1D2D853E85A8012C
:1034D0006B857C858D819E81680F791F89819A819A
:1034E0000E943A1DF7FC11C0A1E0B0E0A219B30997
:1034F0002D893E894F89588D0E94D12DC60ED71E29
:10350000E81EF91E91E0291A3108D301C20122E018
:10351000880F991FAA1FBB1F2A95D1F7880D991DE7
:10352000AA1DBB1DC80ED91EEA1EFB1EAD81BE81A1
:103530001196BE83AD832F85388949895A89420EF9
:10354000531E641E751E9FCF6E960FB6F894DEBF95
:103550000FBECDBFDF91CF911F910F91FF90EF90E4
:10356000DF90CF90BF90AF909F908F907F906F90A3
:103570005F904F903F902F900895CF92DF92EF92FF
:10358000FF920F931F93CF93DF936C017A018B010E
:10359000C0E0D0E0CE15DF0589F0D8016D918D0136
:1035A000D601ED91FC910190F081E02DC6010995C5
:1035B000892B11F47E0102C02196ECCFC701DF9167
:1035C000CF911F910F91FF90EF90DF90CF900895D2
:1035D000089580E090E00895FC01538D448D252FDF
:1035E00030E0842F90E0821B930B541710F0CF969D
:1035F000089501970895FC01918D828D981761F0CF
:10360000828DDF01A80FB11D5D968C91928D9F5F19
:103610009F73928F90E008958FEF9FEF0895FC01C4
:10362000918D828D981731F0828DE80FF11D858D77
:1036300090E008958FEF9FEF0895FC01918D228D0A
:10364000892F90E0805C9F4F821B91098F7399278F
:10365000089580E592E00E941D1B21E0892B09F46A
:1036600020E0822F0895FC01848DDF01A80FB11D99
:10367000A35ABF4F2C91848D90E001968F739927A8
:10368000848FA689B7892C93A089B1898C91806495
:103690008C93938D848D981306C00288F389E02D56
:1036A00080818F7D80830895EF92FF920F931F9307
:1036B000CF93DF93EC0181E0888F9B8D8C8D9813E5
:1036C00005C0E889F989808185FD24C0F62E0B8D1F
:1036D00010E00F5F1F4F0F731127E02E8C8DE81243
:1036E0000CC00FB607FCFACFE889F989808185FF05
:1036F000F5CFCE010E94331BF1CF8B8DFE01E80F79
:10370000F11DE35AFF4FF0820B8FEA89FB8980811C
:10371000806207C0EE89FF896083E889F98980812A
:103720008064808381E090E0DF91CF911F910F91C1
:10373000FF90EF900895CF93DF93EC01888D88235D
:10374000C9F0EA89FB89808185FD05C0A889B9890E
:103750008C9186FD0FC00FB607FCF5CF808185FFE9
:10376000F2CFA889B9898C9185FFEDCFCE010E9457
:10377000331BE7CFDF91CF91089580E090E0892B54
:1037800029F00E94291B81110C94000008950E94C9
:10379000ED2D1F920F920FB60F9211242F933F938E
:1037A0004F935F936F937F938F939F93AF93BF9349
:1037B000EF93FF9380E592E00E94331BFF91EF911E
:1037C000BF91AF919F918F917F916F915F914F9139
:1037D0003F912F910F900FBE0F901F9018951F9241
:1037E0000F920FB60F9211242F938F939F93EF9305
:1037F000FF93E0916002F09161028081E0916602A6
:10380000F091670282FD12C09081809169028F5F02
:103810008F7320916A02821751F0E0916902F0E003
:10382000E05BFD4F958F8093690201C08081FF911D
:10383000EF919F918F912F910F900FBE0F901F903E
:103840001895CF92DF92EF92FF920F931F93CF9331
:10385000DF93D82EC92EF62EE72E8A01E90180913A
:103860002F02882309F48DC060E0809106010E9438
:10387000EF1160E0809107010E94EF118AE28EBD96
:1038800000960096009601D001C0089561E08091F5
:1038900006010E94EF11CEBC0000009601D001C0CD
:1038A00008958FEF9FEF90932C0280932B02DEBC44
:1038B0000000009601D001C00895809129029091E6
:1038C0002A020817190791F01EBD0000009601D0CA
:1038D00001C00895000010932A02009329020EBD32
:1038E00000000096009601D001C0089560E080912C
:1038F00006010E94EF118BE28EBD009600960096A5
:1039000001D001C0089561E0809106010E94EF118D
:10391000EEBC0000009601D001C008958FEF9FEF2C
:1039200090932E0280932D02FEBC0000009601D0E1
:1039300001C008958091270290912802C817D907E5
:1039400091F0DEBD0000009601D001C00895000096
:10395000D0932802C0932702CEBD000000960096A7
:1039600001D001C0089560E0809106010E94EF112E
:103970008CE28EBD00000096009601D001C0089533
:1039800026C08AE20E9422238C2D0E940D238D2DB9
:103990000E940D23812F0E940D23802F0E940D2352
:1039A0008BE20E9422238E2D0E940D238F2D0E94D8
:1039B0000D238D2F0E940D238C2F0E940D238CE24E
:1039C0000E94222360E0809107010E94EF1161E0D4
:1039D00080910601DF91CF911F910F91FF90EF90A1
:1039E000DF90CF900C94EF11CF92DF92EF92FF9285
:1039F0000F931F93CF93DF937A01E901215031098F
:103A0000260F371F41505109480F591F0E94211C92
:103A1000209719F1670180912F02882391F0C70147
:103A2000009771F01EBD02D001D001C008950000C2
:103A30000EBD0096009601D001C00895019791F740
:103A40000AC01C141D043CF4C8010E94372381E005
:103A5000C81AD108F6CF2197DBCF61E0809107012A
:103A6000DF91CF911F910F91FF90EF90DF90CF905A
:103A70000C94EF11EF92FF920F931F93CF93DF936C
:103A8000EA01122F032F41505109480F591F9B0182
:103A90000E94211C7E0180912F02882389F02097AB
:103AA00071F00EBD02D001D001C0089500001EBD0E
:103AB0000096009601D001C00895219791F70BC0A0
:103AC0001E141F0444F4812F902F0E94372381E09D
:103AD000E81AF108F5CF61E080910701DF91CF91FD
:103AE0001F910F91FF90EF900C94EF11EF92FF92C6
:103AF0000F931F93CF93DF93EC018B01F42EE52EF0
:103B00008091170190911801C817D90708F0D1C00A
:103B10008091190190911A016817790708F0C9C0BE
:103B200060E0809107010E94EF1180912F028823AD
:103B300009F493C080912B0290912C028C179D0761
:103B400009F42DC060E0809106010E94EF118AE225
:103B50008EBD0000009601D001C00895D0932C02C4
:103B6000C0932B0261E0809106010E94EF11DEBD3F
:103B700002D001D001C008950000CEBD02D001D016
:103B800001C008950000DEBD02D001D001C008953B
:103B90000000CEBD0000009601D001C008958091C4
:103BA0002D0290912E028017910709F42EC060E03B
:103BB000809106010E94EF118BE28EBD00000096FD
:103BC00001D001C0089510932E0200932D0261E0F0
:103BD000809106010E94EF111EBD02D001D001C0EC
:103BE000089500000EBD02D001D001C0089500006C
:103BF0001EBD02D001D001C0089500000EBD00001E
:103C00000096009601D001C0089560E08091060101
:103C10000E94EF118CE28EBD00960096009601D0B6
:103C200001C0089561E0809106010E94EF11EEBC91
:103C300000960096009601D001C00895D0932A0204
:103C4000C0932902FEBC0000009601D001C0089577
:103C5000109328020093270221C09801AE01B801F9
:103C6000CE010E94211C80912F02811105C08F2D51
:103C70009E2D0E94372312C0E1E0F0E0309771F0F2
:103C8000EEBC02D001D001C008950000FEBC009639
:103C9000009601D001C00895319791F761E08091BD
:103CA0000701DF91CF911F910F91FF90EF900C943E
:103CB000EF11DF91CF911F910F91FF90EF90089539
:103CC0002F923F924F925F926F927F928F929F922C
:103CD000AF92BF92CF92DF92EF92FF920F931F931A
:103CE000CF93DF9300D000D0CDB7DEB77A011801B3
:103CF0004817590720F46C01C41AD50A03C06A0199
:103D0000C81AD90A2617370790F45B01A21AB30A1A
:103D1000CA14DB040CF066C0562F472FB701E52EFE
:103D2000F42E582F492FC901252F342F11C05901C6
:103D3000A61AB70ACA14DB040CF06CC05E2D4F2D16
:103D40007901252F342F582F492FCB01652F742F40
:103D500066246394712C45019594879462177307C8
:103D600018F02FEF3FEF53C0E1E0F0E0FA83E98372
:103D70002B019C838B83EB81FC81EE16FF0608F4FC
:103D800067C040911601423090F050E04150510917
:103D900081019A016114710421F4B2018B819C812B
:103DA00003C06B817C81C2010E943A190DC0A10140
:103DB0006114710421F4B2018B819C8103C06B8179
:103DC0007C81C2010E94761D8C189D0897FE06C05A
:103DD00029813A81420E531E8A0C9B1C8B819C8147
:103DE0000196C7CFE816F90658F5460195948794D1
:103DF0005C2D4D2D6501A52EB42EB901382F292F2C
:103E0000C701E32EF22E612C712C21E030E03A83C1
:103E10002983AECFE816F90698F446019594879465
:103E20005C2D4D2D6501A52EB42EB901382F292FFB
:103E3000C701E32EF22E612C712CEFEFFFEF96CF2E
:103E40005A2D4B2D5601C52ED42E612C712C83CFAB
:103E50000F900F900F900F90DF91CF911F910F91C6
:103E6000FF90EF90DF90CF90BF90AF909F908F909A
:103E70007F906F905F904F903F902F9008950F9399
:103E80001F93E0911601E23058F089014150510929
:103E9000480F591F9B010E94601E1F910F910895AA
:103EA0001F910F910C943A1DEF92FF920F931F9365
:103EB000CF93DF93EA01890120911601FA0131972E
:103EC000223068F09F01260F371FAC010E94601E50
:103ED000DF91CF911F910F91FF90EF9008959F0177
:103EE000260F371FAC010E94211C7E0180912F02FA
:103EF000882389F0209771F01EBD02D001D001C047
:103F0000089500000EBD0096009601D001C00895EE
:103F1000219791F70AC01E141F043CF4C8010E94A7
:103F2000372381E0E81AF108F6CF61E080910701BC
:103F3000DF91CF911F910F91FF90EF900C94EF11B3
:103F4000AF92BF92CF92DF92EF92FF920F931F93A7
:103F5000CF93DF937C016B01EA01590198010E9424
:103F60003F1FB501615071096C0D7D1D9801AE01B7
:103F7000C7010E943F1F9801A501B601C7010E9419
:103F8000541FCE0101979801A501B6018E0D9F1D0A
:103F9000DF91CF911F910F91FF90EF90DF90CF9025
:103FA000BF90AF900C94541FEF92FF920F931F930A
:103FB000CF93DF93EC018B017A0180912F0288234C
:103FC00009F492C08091170190911801C817D90780
:103FD00008F093C08091190190911A016817790730
:103FE00008F08BC060E0809107010E94EF11809182
:103FF0002B0290912C028C179D0711F160E08091AB
:1040000006010E94EF118AE28EBD00000096009624
:1040100001D001C00895D0932C02C0932B0261E01F
:10402000809106010E94EF11DEBD02D001D001C0D7
:1040300008950000CEBD0000009601D001C0089593
:1040400080912D0290912E028017910719F160E066
:10405000809106010E94EF118BE28EBD0000009658
:10406000009601D001C0089510932E0200932D02F6
:1040700061E0809106010E94EF111EBD02D001D0C7
:1040800001C0089500000EBD00000096009601D00A
:1040900001C0089560E0809106010E94EF118CE25A
:1040A0008EBD00960096009601D001C0089561E093
:1040B000809106010E94EF11FEBC02D001D001C028
:1040C00008950000EEBC00000096009601D001C0EB
:1040D000089561E080910701DF91CF911F910F91C9
:1040E000FF90EF900C94EF11CE01DF91CF911F91D3
:1040F0000F91FF90EF900C94761DDF91CF911F915F
:104100000F91FF90EF9008952F923F924F925F9200
:104110006F927F928F929F92AF92BF92CF92DF92D7
:10412000EF92FF920F931F93CF93DF93CDB7DEB73C
:1041300027970FB6F894DEBF0FBECDBF4C015B01D1
:104140008A011901FA018491DA011196FD01449165
:10415000C8010296B8016C5F7F4F98012D5F3F4FF9
:1041600050912F02F80147FF4DC00491602E712C31
:10417000FD01A4917A2AE89477F8FC01849190E0FB
:1041800069837B83F9012491BC01722B7F836E8349
:1041900051110E94151321E000E010E0E12CF12CF8
:1041A00031E0EE81FF81EE16FF060CF07DC0C12CE0
:1041B000D12C27014A0C5B1CC614D704F9F0E98105
:1041C000FB81E983FB830115110529F4049110E0BB
:1041D00023273196F6CF21110BC0A101B201C601F0
:1041E000880D991D2C833D830E94D41F3D812C8115
:1041F000015011097FEFC71AD70ADECF8FEFE81AF7
:10420000F80ACFCF049110E0FD01A491F801FA2B38
:10421000FF83EE83FC01849190E02B01F90124914E
:10422000BC01722B7A83698351110E941513612C92
:10423000712CC12CD12C29813A81C216D306A4F548
:1042400000E010E096012A0D3B1D6E817F8106176C
:104250001707FCF4C801860D971D87709927892BD5
:1042600031F4C2010196F201E490F12C2C01E7FC3B
:104270000BC0A101B901C801880D991D2C833D8394
:104280000E94D41F3D812C81EE0CFF1C0F5F1F4F3D
:10429000DCCFCB0177FF02C080E090E0680E791E92
:1042A0007FEFC71AD70AC7CF27960FB6F894DEBF9D
:1042B0000FBECDBFDF91CF911F910F91FF90EF9077
:1042C000DF90CF90BF90AF909F908F907F906F9036
:1042D0005F904F903F902F90089590912F029923D7
:1042E00059F09CB5209126022CBD8EBD00000DB466
:1042F00007FEFDCF9CBD08950C94CC094F925F92B0
:104300006F927F928F929F92AF92BF92CF92DF92E5
:10431000EF92FF920F931F93CF93DF93EC015B011A
:10432000442E49016801370132E0F32EF092160164
:104330000FEF1FEF21E630E04CE550E067E870E05A
:104340000E94A01F552453945092160184012DE51C
:1043500030E048E550E069E870E0CE0102960E9446
:10436000F41CF09216014E018DE1880E911C00E0C4
:1043700010E021E230E041E250E06BEB70E0C4017C
:104380000E94A01F509216010FEF1FEF2DE130E0A9
:104390004DE150E06DEB70E0CE014F960E94F41CB1
:1043A0004420D1F0F092160100E010E02BED30E057
:1043B0007E018DE3E80EF11CA7016BEB70E0C401F8
:1043C0000E94601E2BEB30E0A7016BED70E0C40192
:1043D0000E94601E50921601109204011092440235
:1043E0001092430286E990E090934202809341024A
:1043F00040E050E066E574E0C5010E94221981E0CA
:104400008093040120914302309144028CE590E0B6
:10441000821B930B97FD0196959587958C0F9D1F99
:10442000909344028093430286E990E09093420285
:104430008093410240E050E066E574E0C5010E94CF
:104440002219C114D10449F020E030E0A60169E945
:1044500070E0CE0108960E94842061147104C9F0B6
:1044600020E030E0A30169E970E0CE01C796DF915A
:10447000CF911F910F91FF90EF90DF90CF90BF9061
:10448000AF909F908F907F906F905F904F900C9423
:104490008420DF91CF911F910F91FF90EF90DF90DB
:1044A000CF90BF90AF909F908F907F906F905F90D4
:1044B0004F900895CF92DF92EF92FF920F931F9348
:1044C000CF93DF93EC0100EF17E823E430E049E2FB
:1044D00050E06CE270E08BE890E00E94F41C26E073
:1044E00030E046E050E06BE270E081E990E00E944D
:1044F0003A1926E030E046E050E06BE270E08DEAE9
:1045000090E00E943A1926E030E046E050E06FE685
:1045100070E081E990E00E943A1926E030E046E040
:1045200050E06FE670E08DEA90E00E943A192CE0CE
:1045300030E04BE150E065E270E082E990E00E94FB
:10454000F41C2CE030E04BE150E06AE670E082E9D8
:1045500090E00E94F41C7E0101E310E023E8C22EEB
:10456000D12CF7018081882399F0D0924402C09227
:10457000430210934202009341024FEF5FEF6BEA58
:104580007BE081917F010E940E18065F1F4FE9CFEB
:1045900001E310E099EBE92EF12C8881882391F05A
:1045A000F0924402E09243021093420200934102CF
:1045B0004FEF5FEF6BEA7BE089910E940E18065F78
:1045C0001F4FEBCFCFE8D0E083EEE82E81E0F82E4E
:1045D00001E310E0F70181917F01882389F0D093F6
:1045E0004402C0934302109342020093410240E010
:1045F00050E06BEA7BE00E940E18065F1F4FEACF87
:104600006C96C33ED10501F7DF91CF911F910F91B9
:10461000FF90EF90DF90CF900895CF93C82F61E087
:10462000809106010E94EF1160E0809107010E94D5
:10463000EF118C2F0E946D2161E080910701CF91D5
:104640000C94EF11CF93C82F60E0809106010E9477
:10465000EF1160E0809107010E94EF118C2F0E9402
:104660006D2161E080910701CF910C94EF110CB4A2
:1046700005FC0DC09EBD00000DB407FEFDCF9EB52C
:104680008EBD00000DB407FEFDCF8EB508958EBD22
:1046900000000DB407FEFDCF8EB59EBD00000DB429
:1046A00007FEFDCF9EB508952F923F924F925F92E5
:1046B0006F927F928F929F92AF92BF92CF92DF9232
:1046C000EF92FF920F931F93CF93DF93CDB7DEB797
:1046D0002A970FB6F894DEBF0FBECDBF9E838D83A1
:1046E00078876F835A8749875901480188E2682E85
:1046F000712C96E4492E512C24E9222E312C0E9453
:10470000402685E690E09093440280934302EFE0D8
:10471000F0E0F0934202E093410240EE5FEF66E585
:1047200074E08D819E810E942219709244026092F1
:10473000430250924202409241024FEF5FEF66E522
:1047400074E08F8198850E94221930924402209251
:10475000430250924202409241024FEF5FEF66E502
:1047600074E0F501808191810E94C4180FEF1FEF62
:1047700022E230E042E250E060E370E080EB90E063
:104780000E94A01F2FEF3FEF48E254E069E370E082
:1047900085EB90E00E948420709244026092430274
:1047A00088E790E090934202809341024FEF5FEFE1
:1047B00066E574E089859A850E9422193092440248
:1047C00020924302E8E7F0E0F0934202E0934102D6
:1047D0004FEF5FEF66E574E0F401808191810E9404
:1047E000C41822E230E042E250E062E670E080EB82
:1047F00090E00E94A01F2FEF3FEF48E254E06BE6ED
:1048000070E085EB90E00E94842022E230E04DE3EE
:1048100050E066EC70E081E890E00E94A01F2EE17D
:1048200030E049E350E068EC70E083E890E00E94FB
:10483000F41C82E990E090934402809343028CED53
:1048400090E0909342028093410240E050E066E5A0
:1048500074E08BEE91E00E942219BE016F5F7F4FE2
:10486000CE0103960E949713882381F189819A8152
:10487000813A91050CF052C08336910584F0F40121
:10488000808191818E159F051CF48C0D9D1D17C094
:10489000F501808191818C0D9D1DF40110C0C1979F
:1048A000ACF0F50180819181F401208131812C19D6
:1048B0003D098217930734F48C0D9D1DF5019183FA
:1048C00080831DCFF5011182108219CF0E948C12B6
:1048D00000913D0210913E0220913F023091400232
:1048E000DC01CB01801B910BA20BB30B893E9340E3
:1048F000A105B10508F4B1CF60E080E090E00E942E
:104900007910892B69F40E948C1260933D02709398
:104910003E0280933F02909340029FCF80E001C00F
:1049200081E02A960FB6F894DEBF0FBECDBFDF91AF
:10493000CF911F910F91FF90EF90DF90CF90BF909C
:10494000AF909F908F907F906F905F904F903F902F
:104950002F900895EF92FF920F931F93CF93DF93C1
:104960000E94402680E090E00E94F50841E080919E
:10497000340290913502892B09F040E022E8E22EC2
:1049800023E0F22E05ED13E020EF3FEF6EEE71E035
:104990008AE090E00E947E2141E080913402909173
:1049A0003502019709F040E096EBE92E92E0F92EEE
:1049B0000CE113E02FEF37E868E471E082E790E064
:1049C0000E947E2141E0809134029091350202974D
:1049D00009F040E083E1E82E82E0F82E06E612E0DE
:1049E0002FE13CEF68E571E08AED90E00E947E21C6
:1049F000809134029091350281309105E1F1029766
:104A000009F086C08CEF91E00E945A228BE390E07F
:104A10009093440280934302CEE5D0E0D0934202CB
:104A2000C09341024FEF5FEF66E574E086E591E0E9
:104A30000E94221988EC90E09093440280934302F4
:104A4000D0934202C09341024FEF5FEF66E574E0FE
:104A50008FE491E00E9422192FEF3FEF46E652E0EB
:104A60006BE270E080E590E00E9484202FEF3FEF42
:104A700043E152E099C086EF91E00E945A228BE117
:104A800090E09093440280934302CEE5D0E0D0932F
:104A90004202C09341024FEF5FEF66E574E08DE3A1
:104AA00091E00E94221988EC90E090934402809358
:104AB0004302D0934202C09341024FEF5FEF66E59D
:104AC00074E086E491E00E9422192FEF3FEF4AED57
:104AD00051E06BE270E08FE690E00E9484202FEFBF
:104AE0003FEF41EA51E06BE270E083EC90E00E941E
:104AF00084202FEF3FEF4CE153E06BE270E080E564
:104B000090E00E9484202FEF3FEF46EB52E04CC034
:104B100082E092E00E945A2283E590E09093440262
:104B200080934302CEE5D0E0D0934202C09341028D
:104B30004FEF5FEF66E574E089E391E00E94221990
:104B400088EC90E09093440280934302D093420219
:104B5000C09341024FEF5FEF66E574E082EF91E0B2
:104B60000E9422192FEF3FEF4AED51E06BE270E017
:104B70008FE690E00E9484202FEF3FEF41EA51E062
:104B80006BE270E083EC90E00E9484202FEF3FEF17
:104B900045ED53E06BE270E080E590E00E948420F8
:104BA0002FEF3FEF42E853E06BE270E08BED90E0D7
:104BB0000E9484200FEF1FEF2AE130E043E450E031
:104BC00064E070E089EF90E00E94A01F00E114E82B
:104BD00028E130E041E450E065E070E08AEF90E0E9
:104BE0000E94F41C8DEF90E0909344028093430266
:104BF00087E190E0909342028093410240E050E0D0
:104C000066E574E088E092E00E94221984E090E07A
:104C100090934402809343028FE090E0909342028D
:104C2000809341024FE154E866E574E08EE092E043
:104C30000E94221986E090E00E945807EC010E9431
:104C4000EC069B01AC01DE010E94D12D9B01AC0161
:104C5000ABE2B0E00E94C62D20E030E943E350E033
:104C60000E94832DDA01C9014FE154E866E574E042
:104C7000DF91CF911F910F91FF90EF900C94290736
:104C80000F931F932091190130911A014091170140
:104C90005091180100E010E060E070E080E090E0EA
:104CA0000E94F41C1F910F910895009769F0FC0178
:104CB00001900020E9F73197AF01481B590BBC0167
:104CC00080E592E00C94BD1A80E090E008958F9208
:104CD0009F92AF92BF92CF92DF92EF92FF920F938B
:104CE0001F93CF93DF93CDB7DEB7A1970FB6F8949C
:104CF000DEBF0FBECDBF6B017C0197FF31C0E091DD
:104D00005002F09151020190F081E02D6DE280E5BA
:104D100092E009958C0122273327A9012C193D091E
:104D20004E095F0919A2CE0181967C019AE0892E75
:104D3000912CA12CB12CCA01B901A50194010E94AA
:104D4000612D605DF70162937F01211531054105F9
:104D5000510589F7CF010E945526800F911F1DC074
:104D60009B01AC0119A28E010F5D1F4F8AE0C82E76
:104D7000D12CE12CF12CCA01B901A70196010E94A6
:104D8000612D605DF80162938F01211531054105A8
:104D9000510589F7CF010E945526A1960FB6F894C8
:104DA000DEBF0FBECDBFDF91CF911F910F91FF905E
:104DB000EF90DF90CF90BF90AF909F908F9008952D
:104DC000CF93DF93BC01990F880B990B0E94672644
:104DD000EC018AE991E00E9455268C0F9D1FDF911E
:104DE000CF9108950C945526CF93DF930E945526BA
:104DF000EC018AE991E00E9455268C0F9D1FDF91FE
:104E0000CF9108952F923F924F925F926F927F922F
:104E10008F929F92AF92BF92CF92DF92EF92FF92CA
:104E20000F931F93CF93DF93CDB7DEB72E970FB6B7
:104E3000F894DEBF0FBECDBF5C011B016A013E8747
:104E40002D871A87098747018FEF9FEF90934F02B5
:104E500080934E0210924D0210924C0210924B021F
:104E600010924A0280914902882321F08FE891E054
:104E70000E94F42685E0889D9001899D300D1124C3
:104E80003A8329838C9CA0018D9C500D9C9C500DD5
:104E900011245E834D834D855E85C49E9001C59E21
:104EA000300DD49E300D112438872F83849F9001BC
:104EB000859F300D11243C832B83612C712C412C58
:104EC000512C2D853E8549855A85421753070CF490
:104ED000B1C04D855E85452B39F460E180E00E94CC
:104EE000D609C12CD12C3FC08F819885860D971D86
:104EF0006AE070E00E944D2DC101860F971F8F3F21
:104F0000910511F00CF096C060E1E9CF81E090E0EE
:104F10000E9458079C0180E090E02B873C870E940C
:104F20005807AC0181E02B853C85C114D10409F000
:104F300080E0EE24EA9463E0F62E0D851E8561E0A4
:104F40000E948007809147029091480297FF03C01A
:104F5000C12CDD24D39452E0C50ED11C2FEFC21614
:104F6000D10409F07CF461E070E08C2D0E94070A06
:104F7000C114D10459F66EE170E080E090E00E9427
:104F80005212C4CF4D855E8514161506C4F52091C6
:104F90004502309146022F5F3F4F309344022093E9
:104FA00043020296909342028093410252E0A5167A
:104FB000B10499F084E0A816B10409F54FEF5FEF52
:104FC0006BEA7BE08D859E850E9429074FEF5FEF9E
:104FD0006BEA7BE08BE891E010C04FEF5FEF6BEA8C
:104FE0007BE08B819C81840D951D0E94C4184FEF3E
:104FF0005FEF6BEA7BE081E991E00E9422198091EA
:105000004902882321F08DE891E00E94F4260E9455
:10501000150729813A81420E531E4D815E81640E2F
:10502000751E811122C08D859E85880D991D9E87D4
:105030008D8747CFC5012E960FB6F894DEBF0FBE01
:10504000CDBFDF91CF911F910F91FF90EF90DF9037
:10505000CF90BF90AF909F908F907F906F905F9018
:105060004F903F902F900C94130B2E960FB6F89400
:10507000DEBF0FBECDBFDF91CF911F910F91FF908B
:10508000EF90DF90CF90BF90AF909F908F907F90E8
:105090006F905F904F903F902F90089590E0FC01AB
:1050A000E956F44F2491FC01ED57F44F8491882385
:1050B00099F090E0880F991FFC01E758F44FA591F3
:1050C000B491FC01E159F44F859194918FB7F89414
:1050D000EC91E22BEC938FBF0895CF93DF9300D038
:1050E00000D0CDB7DEB7789484B5826084BD84B536
:1050F000816084BD85B5826085BD85B5816085BDD3
:1051000080916E00816080936E001092810080918A
:105110008100826080938100809181008160809312
:105120008100809180008160809380008091B10037
:1051300084608093B1008091B00081608093B00062
:1051400080917A00846080937A0080917A008260F6
:1051500080937A0080917A00816080937A008091B8
:105160007A00806880937A001092C1008DE00E94DE
:105170004E288AE00E944E2810922F0282E08093EF
:10518000070184E08093060183E0809305010E947B
:10519000E21260E083E00E94EF1183E00E944E285B
:1051A00061E084E00E94EF1184E00E944E2861E0FB
:1051B00082E00E94EF1182E00E944E2880E491E09C
:1051C000909318018093170180EF90E090931A015B
:1051D00080931901109244021092430210924202ED
:1051E000109241028FEF9FEF90932E0280932D0239
:1051F00090932C0280932B0290932A028093290291
:1052000090932802809327028CB58C7F8CBD8DB53E
:1052100081608DBD8CB58F7D8CBD8CB5837F8CBD41
:105220008CB58093260210910501112309F493C2D5
:1052300061E0812F0E94EF1165E070E080E090E076
:105240000E94521260E0812F0E94EF1164E170E031
:1052500080E090E00E94521261E0812F0E94EF11E5
:1052600066E970E080E090E00E945212E4E3F1E031
:10527000B49005E311E0BB2009F436C0F801849135
:105280000E9422236801F2E0CF0ED11CF801319672
:105290000491202F2078A22E0F777601102F115025
:1052A00040F0F70184910E940D23FFEFEF1AFF0AEF
:1052B000F6CFC601800F911D8C01AA2099F07C01C8
:1052C0009FEFE91AF90AF80164916F3F21F070E04D
:1052D00080E090E004C064EF71E080E090E00E9424
:1052E00052128701BA94C7CF86E30E94222388EE28
:1052F0000E940D2320E431E030931101209310012E
:105300008CE39FE090930F0180930E0130930D0189
:1053100020930C0190930B0180930A0183E080930A
:10532000090187E0809308010E944E2860E087E031
:105330000E94EF11BE016F5F7F4FCE0103960E9466
:105340009713E0916002F091610282E08083E09126
:105350005C02F0915D021082E0915E02F0915F02CA
:105360008FEC808310926802E0916402F0916502F4
:1053700086E08083E0916202F09163028081806127
:105380008083E0916202F091630280818860808373
:10539000E0916202F0916302808180688083E091F5
:1053A0006202F091630280818F7D808383E691E0C9
:1053B0000E94F4260E94E21280E590E00E94D30948
:1053C00080E090E00E94F90A0E94AA24BB24B394D2
:1053D00080E592E00E941D1B892B09F482C00E9487
:1053E000EA0890E0FC01E154F109EA32F10508F025
:1053F00078C0E45BFF4F0C94A22D0E94EA0862E0A3
:1054000070E00E94070A6BC0B09249020E94EA084D
:1054100062E070E00E94F30962C0B092490282E04B
:1054200090E004C0B092490281E090E00E94B20E88
:1054300056C0B092490284E090E0F8CFB0924902A1
:1054400083E090E0F3CFB092490285E090E0EECFA8
:10545000B092490286E090E0E9CF60E980E00E94E6
:10546000D60962E370E080E00E94F30960E98FEF03
:105470000E94D60962E370E08FEF0E94F309EDCF3E
:10548000B092490288E090E0D1CFB092490287E023
:1054900090E0CCCF0E94EA08182F0E94EA08482F1B
:1054A00050E0612F70E085E090E00E941B0A80E5EB
:1054B00092E00E941D1B892BD1F313C061E080E0B4
:1054C00090E00E9479100E94E02609C0B092360256
:1054D00006C010923802109237020E94AA24B0929D
:1054E000490280913602882309F482C080914902E2
:1054F000882321F087E991E00E94F22680914902F9
:10550000882351F083E090E00E945807BC01990F76
:10551000880B990B0E94672680914902882321F00D
:1055200087E391E00E94F22680914902882351F09E
:1055300082E090E00E945807BC01990F880B990BFC
:105540000E94672680914902882321F087E391E039
:105550000E94F22680914902882351F080E090E079
:105560000E945807BC01990F880B990B0E9467266F
:1055700080914902882321F087E391E00E94F2267E
:1055800080914902882351F081E090E00E94580701
:10559000BC01990F880B990B0E94672680914902E4
:1055A000882321F087E391E00E94F226809149024E
:1055B000882351F087E090E00E945807BC01990FC2
:1055C000880B990B0E94672680914902882321F05D
:1055D00087E391E00E94F22680914902882341F0FE
:1055E0000E94EC060E9467268AE991E00E945526F7
:1055F0000E948C120091390210913A0220913B02D4
:1056000030913C02DC01CB01801B910BA20BB30B50
:10561000893E9340A105B10510F1809149028111A5
:105620001EC0E0903702F090380260E0C7010E948F
:1056300079108C01EF2809F0AAC00115110509F0B5
:1056400092C00E9415078111ACC00E948C12609319
:10565000390270933A0280933B0290933C0280910E
:10566000370290913802892B09F072C0BE016F5F3A
:105670007F4FCE0103960E949713882309F460C0E0
:1056800089819A818937910514F12B813C81809120
:105690003402909135022A3631053CF4892BB9F059
:1056A000109235021092340210C0253D31052CF4C1
:1056B000019769F081E090E004C0029741F082E038
:1056C00090E090933502809334020E94AA2489814D
:1056D0009A81CC97ACF58B819C81863D910584F1B4
:1056E000809134029091350201970297B8F4CC244E
:1056F000C394D12C3CE0E32EF12C02E111E020E335
:1057000032E04DE951E068EA71E083EB91E00E94FC
:105710005423811115C00E94AA2412C082E3C82E0E
:10572000D12C9EE5E92EFF24F39404E111E022E35D
:1057300032E04FEB51E06AEC71E085ED91E0E7CFAC
:1057400080914902811104C080E090E00E94F90A32
:105750000E94BD1B3DCE81E00E9422236AE070E0E2
:1057600080E090E081CD64EF71E080E090E00E9405
:10577000521261E0C8010E9479108C01009711F06B
:105780000E94B20E10933802009337025ACF012BB9
:1057900009F057CF0E94AA241092380210923702C3
:1057A00050CF8091370290913802892B09F44DCF68
:1057B0000E94AA24109238021092370246CFE0E5E8
:1057C000F2E01382128288EE93E0A0E0B0E08483DE
:1057D0009583A683B7838FE191E09183808385ECE5
:1057E00090E09587848784EC90E09787868780ECAB
:1057F00090E0918B808B81EC90E0938B828B82EC9C
:1058000090E0958B848B86EC90E0978B868B118E45
:10581000128E138E148E08955058BB27AA270E940B
:10582000242C0C94032D0E94F52C38F00E94FC2CA3
:1058300020F039F49F3F19F426F40C94F22C0EF466
:10584000E095E7FB0C94EC2CE92F0E94142D58F303
:10585000BA17620773078407950720F079F4A6F555
:105860000C94362D0EF4E0950B2EBA2FA02D0B01C3
:10587000B90190010C01CA01A0011124FF27591B95
:1058800099F0593F50F4503E68F11A16F040A22F9B
:10589000232F342F4427585FF3CF4695379527950C
:1058A000A795F0405395C9F77EF41F16BA0B620B0B
:1058B000730B840BBAF09150A1F0FF0FBB1F661F52
:1058C000771F881FC2F70EC0BA0F621F731F841F95
:1058D00048F4879577956795B795F7959E3F08F0BB
:1058E000B0CF9395880F08F09927EE0F979587957D
:1058F00008950E94802C6894B1110C94372D08955E
:105900000E941C2D88F09F5798F0B92F9927B75106
:10591000B0F0E1F0660F771F881F991F1AF0BA9553
:10592000C9F714C0B13091F00E94362DB1E008954E
:105930000C94362D672F782F8827B85F39F0B93F40
:10594000CCF3869577956795B395D9F73EF4909506
:105950008095709561957F4F8F4F9F4F0895E89484
:1059600009C097FB3EF490958095709561957F4FA7
:105970008F4F9F4F9923A9F0F92F96E9BB27939555
:10598000F695879577956795B795F111F8CFFAF465
:10599000BB0F11F460FF1BC06F5F7F4F8F4F9F4F96
:1059A00016C0882311F096E911C0772321F09EE8F4
:1059B000872F762F05C0662371F096E8862F70E05A
:1059C00060E02AF09A95660F771F881FDAF7880F34
:1059D0009695879597F9089597F99F6780E870E005
:1059E00060E008959FEF80EC089500240A94161655
:1059F000170618060906089500240A9412161306BD
:105A0000140605060895092E0394000C11F488234A
:105A100052F0BB0F40F4BF2B11F460FF04C06F5F66
:105A20007F4F8F4F9F4F089557FD9058440F551F3C
:105A300059F05F3F71F04795880F97FB991F61F010
:105A40009F3F79F087950895121613061406551F87
:105A5000F2CF4695F1DF08C0161617061806991FF3
:105A6000F1CF86957105610508940895E894BB27E8
:105A700066277727CB0197F90895DB018F939F93D2
:105A80000E94C62DBF91AF91A29F800D911DA39F33
:105A9000900DB29F900D1124089597FB072E16F4D8
:105AA000009407D077FD09D00E94D92D07FC05D0BE
:105AB0003EF4909581959F4F0895709561957F4F25
:105AC0000895A1E21A2EAA1BBB1BFD010DC0AA1F3F
:105AD000BB1FEE1FFF1FA217B307E407F50720F057
:105AE000A21BB30BE40BF50B661F771F881F991FD2
:105AF0001A9469F760957095809590959B01AC011B
:105B0000BD01CF010895052E97FB1EF400940E945D
:105B10009A2D57FD07D00E94612D07FC03D04EF44B
:105B20000C949A2D50954095309521953F4F4F4FAD
:105B30005F4F089590958095709561957F4F8F4F39
:105B40009F4F0895EE0FFF1F0590F491E02D0994EB
:105B50000E94B02D332312F48A1B9B0B0C94C12D91
:105B6000A29FB001B39FC001A39F700D811D11249E
:105B7000911DB29F700D811D1124911D08950E94E9
:105B8000B02DB7FF0895821B930B08950E94B02D8E
:105B9000A59F900DB49F900DA49F800D911D112481
:105BA0000895B7FF0C94C62D0E94C62D821B930B3F
:105BB0000895AA1BBB1B51E107C0AA1FBB1FA61754
:105BC000B70710F0A61BB70B881F991F5A95A9F7A6
:105BD00080959095BC01CD01089581E090E0F89406
:085BE0000C94F22DF894FFCFA4
:105BE800FF0000000107080A02013C0F40013C0FBA
:105BF80040010C005E01014001F00000000000546B
:105C08001BBD1AEC1A9B1B1D1BFB1A0F1B2D002E0C
:105C1800006D20006C20002C00504E5000702D4D5F
:105C28004F53464554006E2D4D4F53464554007012
:105C38002D4A464554006E2D4A4645540044696F26
:105C480064650043757276652054726163657200FD
:105C5800206761696E3D0067203000205674683DFA
:105C68000020566F66663D0067200056007A006E79
:105C7800007541006D41007820000D0A004D6178E3
:105C880020562D67617465004D696E20562D676139
:105C98007465002020464554205365747570004D86
:105CA800617820492D62617365004D696E20492D28
:105CB80062617365004269706F6C6172205365742C
:105CC8007570006F6F6F6F6F6F6F004F4B00504EA6
:105CD80050204E504E0073676473670064677364A6
:105CE8006700656263656200534554555000426120
:045CF8007420000014
:00000001FF
